:020000020000FC
:100000000C9490030C94A0050C948D050C94900313
:100010000C9490030C9490030C946B030C94900339
:100020000C9490030C9490030C9490030C94900304
:100030000C9490030C9490030C9490030C949003F4
:100040000C9496050C9490030C9490030C949003DC
:100050000C9490030C9490030C9490030C949003D4
:100060000C9490030C949003475053444F205954E0
:100070002076312E30200400436F756E74730400B7
:100080004F736320686561742D75702077616974A2
:100090002031356D04005075736820627574746F7B
:1000A0006E20746F2070617373200400576169744F
:1000B000696E672E2E2E040043616C696272617452
:1000C000696F6E2070686173652031200400436F92
:1000D000756E74696E672E2E2031732073616D709A
:1000E0006C65040043616C6962726174696F6E20B3
:1000F0007068617365203220040043616C6962722C
:100100006174696F6E20706861736520332004002C
:1001100043616C6962726174696F6E2070686173AB
:10012000652034200400436F756E74696E672E2E4F
:100130003630732073616D706C650400436F756EAB
:1001400074696E672E2E3130732073616D706C652B
:100150000400436F756E74696E672E323030732001
:1001600073616D706C650400736C6F77696E672DD9
:10017000646F776E2E2E2E2004007370656564699F
:100180006E672D75702E2E2E20200400417765732A
:100190006F6D65203A292020202020200400202097
:1001A000202020202020202020202020202020204F
:1001B000202004004E6F2070756C73652064657498
:1001C0006563746564202020040053656C662072AA
:1001D000756E6E696E67206D6F64652E2E2E04003D
:1001E0005265736574696E672064656661756C74C9
:1001F0002E2E2E200400656570726F6D20636F6E69
:1002000066696720666F756E642004004E6F206318
:100210006F6E66696720666F756E642C20353025B9
:10022000040070776D2073657420746F20646566B8
:1002300061756C74202004005365742070776D2004
:10024000546F3A203078040043616C6962726174C3
:10025000696F6E2070686173652035200400436FFC
:10026000756E74696E672E393030732073616D70EE
:100270006C65040052756E6E696E67206D6F646503
:100280002E2E2E20202020200400436F756E7469CE
:100290006E672031302042696C6C696F6E200400FB
:1002A00030313233343536373839414243444546AC
:1002B00003E008B91ED003E008B91BD003E008B979
:1002C00018D002E008B915D002E008B912D093D0D6
:1002D00008E008B90ED000E008B90BD00CE008B96E
:1002E00008D000E008B905D006E008B902D00BD06C
:1002F00008954598449A7FD044980895459A449A21
:1003000074D04498089500E008B9F3DF01E008B91B
:10031000F0DF089508E008B9ECDF00E008B9E9DF94
:1003200008950CE008B9E5DF00E008B9E2DF0895C0
:1003300009E008B9DEDF04E008B9DBDF08950DE06D
:1003400008B9D7DF04E008B9D4DF089500E205D08A
:100350000895F1E0EEE939D00895102F02950F705D
:100360001F7008B9CBDF18B9C9DF089500932101C8
:1003700013E018B9C3DF0091210110EF01230295AA
:1003800008B9BCDF13E018B9B9DF009121011FE003
:10039000012308B9B3DF08950093210113E018B9D0
:1003A000ADDF0091210110EF0123029508B9A6DF0E
:1003B00008950093210113E018B9A0DF00912101F5
:1003C0001FE0012308B99ADF0895C895002D043075
:1003D00059F0002D102D02950F701F7008B98EDF97
:1003E00018B98CDF3196F1CF089526EA2A95F1F7F6
:1003F00000000000089531E229EC2A95F1F73A95C2
:10040000D9F700000000089585DFF0E0E8EBDDDFBC
:1004100088DFF0E0EEECD9DF08957CDFF0E0E4EE79
:10042000D4DF7FDFF1E0ECE3D0DF089573DFF0E0AD
:10043000EAEFCBDF76DFF1E0E6E2C7DF08956ADFBF
:10044000F1E0E0E1C2DF6DDFF1E0E2E5BEDF08955B
:1004500061DFF2E0E8E4B9DF64DFF2E0EEE5B5DFAA
:10046000089558DFF2E0E4E7B0DF5BDFF2E0EAE8AE
:10047000ACDF089564DFF1E0E8E6A7DF08955FDF11
:10048000F1E0EAE7A2DF08955ADFF1E0ECE89DDF52
:1004900008950F9302950F70F2E0E0EAE00F08F480
:1004A000F395C895002D59DF0F910F70F2E0E0EA47
:1004B000E00F08F4F395C895002D4FDF08958827C5
:1004C000579F402C512C469F202C312C569F300C8E
:1004D000411C581E479F300C411C581E0895400F68
:1004E000511F621F731F0895112722273327BB272F
:1004F000AA279927881BC1E2779567955795479555
:10050000CA9551F020F4800F911FA21FB31FB79519
:10051000A79597958795F0CF089500271127222753
:100520003327442755276627772788279927AA271F
:10053000BB27CC27DD27EE27FF270895A89572E477
:1005400086ED9BEE9A95F1F78A95D9F77A95C1F7E2
:1005500073E07A95F1F700000895DD27CC2701E0DC
:1005600000930201EBDFA89500910201003021F019
:100570002196CA17DB07B1F70027009302010895FF
:10058000DD27CC2755276627772788279927C8E2B4
:100590000ED0000F111F221F331F441F551F661F4F
:1005A000771F881F991FAA1FCA9591F708955F9317
:1005B0005F70553010F05D5FD52FD52F5F91507F64
:1005C000503508F0505D5D0F6F936F70653010F01F
:1005D0006D5FD62FD62F6F91607F603508F0605D1C
:1005E0006D0F7F937F70753010F07D5FD72FD72F01
:1005F0007F91707F703508F0705D7D0F8F938F70E5
:10060000853010F08D5FD82FD82F8F91807F803567
:1006100008F0805D8D0F9F939F70953010F09D5F67
:10062000D92FD92F9F91907F903508F0905D9D0F25
:100630000895AF93AF70A53010F0AD5FDA2FDA2FC9
:10064000AF91A07FA03508F0A05DAD0F0895F99996
:10065000FECF112711BD12BDF1E0EBE2019100BD0B
:1006600004E00FBBFA9AF99AF999FECF139511BDE0
:100670001230A1F711270895F999FECF11270091A3
:1006800034010F3F19F402E000933401112712BD29
:1006900001BDF1E0E9E0019100BD04E00FBBFA9A71
:1006A000F99AF999FECF139511BD1130A1F708956C
:1006B000F999FECFAA27BB27A1BDB2BDF1E0EBE2BD
:1006C000F89AF899FECF00B501931196A1BDB2BD7D
:1006D000A230B1F70895A89501E000932D0113DE33
:1006E00019DEF1E0E4EB71DE1CDEF1E0EAEC6DDE38
:1006F00001E005BB00E005BD10DF06BD0093000171
:100700000093010127C3BB27AA27F999FECFB2BDE9
:10071000A1BD0FEF00BDFA9AF99AA395B1F708951C
:100720000FEF0DBF08E00EBF02E0009334010FEFA2
:1007300004B907B900270AB908B90FEF0BB902E0ED
:100740000DBB0BE000936900B3DD4B9909C0DBDD05
:10075000E1DDF1E0E0EE39DED6DFBB27A5E0FDDE2E
:100760000FEF009387000FEF0093860002E80093DD
:10077000800009E1009381009BDF10912C01209102
:100780002B010FEF10172007F1F000912B010093C0
:10079000890000912C0100938800B5DDBBDDF1E0FC
:1007A000E6EF13DEBEDDF2E0E8E30FDE00912B01A1
:1007B00070DE00912C016DDEBB27A5E0CEDE05E0EA
:1007C0000093030115C00FE7009389000FEF00931A
:1007D000880099DD9FDDF2E0ECE0F7DDA2DDF2E0DC
:1007E000E2E2F3DDBB27A5E0B8DE01E00093030100
:1007F00001E000936E0000E005BD002706BD0093F8
:100800000001009301018ED288DEA89508E10093D3
:10081000600006E40093600000910301053041F0A0
:1008200001E000932E01002700932F01EDDD92C21D
:100830000FDE04E800932E0103E000932F018AC22B
:10084000E3DD00910901003869F0EAF013DE309130
:100850008900209188002D533A40309389002093DD
:10086000880078C211DEB0E0A5E077DE68DD71DDDA
:10087000D4DD02E0009303010AE000932E0100277B
:1008800000932F0167C2FBDDB0918900A091880021
:100890000DE31AE0A00FB11FB0938900A093880068
:1008A00059C2BBDD0AE000932E01002700932F01FF
:1008B00000910901003091F0009109010233F8F034
:1008C000DEDDB0918900A091880006E011E0A00F64
:1008D000B11FB0938900A09388003CC2D5DDB0E081
:1008E000A5E03BDE2CDD35DDA1DD03E00093030157
:1008F0000CE300932E01002700932F012BC2BADDD9
:100900003091890020918800265031403093890031
:10091000209388001FC28ADD0CE300932E0100277C
:1009200000932F0100910901003081F00F37F8F09A
:10093000A6DDB0918900A09188000BE210E0A00F25
:10094000B11FB0938900A093880004C29DDDB0E080
:10095000A5E003DE74DDF3DCFCDC04E000930301BE
:1009600008EC00932E01002700932F01F3C182DDD4
:1009700030918900209188002B52304030938900BB
:1009800020938800E7C15BDD08EC00932E0100276F
:1009900000932F0100910901003081F00F37F8F02A
:1009A0006EDDB0918900A09188000CE010E0A00FEE
:1009B000B11FB0938900A0938800CCC165DDB0E081
:1009C000A5E0CBDD45DDBBDCC4DC05E00093030125
:1009D00004E800932E0103E000932F01BBC14ADD20
:1009E00030918900209188002C503040309389004C
:1009F00020938800AFC12CDD3FDE009134010395C8
:100A00000093340104E800932E0103E000932F01CA
:100A100000910901003089F00F3770F030DDB0919E
:100A20008900A091880003E010E0A00FB11FB093EF
:100A30008900A09388008EC11AC026DD30918900FC
:100A40002091880030932B0120932C0100DEB0E030
:100A5000A5E083DD06DD73DC7CDC06E000930301AA
:100A600008EE00932E0103E000932F0173C102DD15
:100A7000B0918900A0918800A350B040B093890044
:100A8000A093880067C100910901F6DD009134014F
:100A9000039500933401E5DC08EE00932E0103E09A
:100AA00000932F0100910901003089F00F3770F099
:100AB000E6DCB0918900A091880002E010E0A00F70
:100AC000B11FB0938900A093880044C11AC0DCDC38
:100AD000309189002091880030932B0120932C01C4
:100AE000B6DDB0E0A5E039DDBCDC29DC32DC06E0B7
:100AF0000093030108EE00932E0103E000932F0101
:100B000029C1B8DCB0918900A0918800A250B04002
:100B1000B0938900A09388001DC1009102010130AB
:100B200021F4002700930201189518950FEFA017E4
:100B3000B00711F0119618952196AA27BB27189592
:100B4000009101011091000120912F0130912E019F
:100B50001317020769F0A89501E005BDF0910101A6
:100B6000E09100013196F0930101E09300011895A6
:100B700000E005BD00270093010100930001A89546
:100B80005B2F4A2F71E060E09ADC2F923F924F92E8
:100B90005F92DF93CF93C1DCCF91DF914C2F5D2F1C
:100BA00031E0A5DC3F912F911F910F919927400FC4
:100BB000511F621F731F891F06B511272227332774
:100BC0009927400F511F621F731F891FA89B0CC0DC
:100BD00001E005BB002711E0222733279927400FAA
:100BE000511F621F731F891F4093090150930A010F
:100BF00060930B0170930C0180930D0140910D01E6
:100C000030910C0120910B0110910A010091090112
:100C1000B7DC5093220160932301709324018093E9
:100C2000250190932601A093350182DB92DB80DBC6
:100C3000009103010630A1F00091260197DB00919D
:100C4000250194DB0091240191DB009123018EDBCF
:100C5000009122018BDB7ADBF0E0E8E7B6DB29C00C
:100C600000913501003011F471DB03C000913501B2
:100C7000A0DB0091260190DB0CE26FDB00912601E6
:100C800098DB0091250172DB0CE267DB0091240107
:100C90006DDB0091230180DB0EE25FDB009123011D
:100CA00088DB0091220162DB51DB08E456DB0AE7B6
:100CB00054DB33DC06BD0093000100930101009179
:100CC0000301013031F40FEF0DBF08E00EBFF894BF
:100CD000B7CD023031F40FEF0DBF08E00EBFF8942E
:100CE000E0CD033031F40FEF0DBF08E00EBFF894F4
:100CF00012CE043031F40FEF0DBF08E00EBFF894B0
:100D000042CE053031F40FEF0DBF08E00EBFF8946E
:100D100072CE063031F40FEF0DBF08E00EBFF8942D
:100D2000B2CE1895F0DAF6DAF0E0E8E64EDBF9DA62
:100D3000F0E0E0E84ADBFCDAF0E0E6E946DBFFDA87
:100D4000F0E0ECEA42DBA8957894B3E0A4E805DC97
:100D5000DADA0895F3DBF2DBE0DB01E00CBB01E063
:100D60000DBBA89578940000000000000000000072
:100D70000000000000000000000000000000000073
:100D80000000000000000000000000000000000063
:100D90000000000000000000000000000000000053
:100DA0000000000000000000000000000000000043
:0A1D200000000000000000001EC8D3
:00000001FF
